:020000040000FA
:04000000C9EF05F04F
:080008005DEF00F000000000B4
:100010000000000000000000056ED8CF06F0E0CF21
:1000200007F00001E9CF0DF0EACF08F0E1CF09F0C9
:10003000E2CF0AF0D9CF0BF0DACF0CF0F3CF14F007
:10004000F4CF15F0FACF16F000C00FF001C010F099
:1000500002C011F003C012F004C013F09DA034EFF1
:1000600000F09EB0BDEF00F09DA23AEF00F09EB20E
:100070009AEF04F00FC000F010C001F011C002F0C0
:1000800012C003F013C004F00E8E0DC0E9FF08C0CB
:10009000EAFF09C0E1FF0AC0E2FF0BC0D9FF0CC0B4
:1000A000DAFF14C0F3FF15C0F4FF16C0FAFF0550C5
:1000B00007C0E0FF06C0D8FF10000001E9CF1EF026
:1000C000EACF19F0E1CF1AF0E2CF1BF0D9CF1CF044
:1000D000DACF1DF0F3CF25F0F4CF26F0FACF27F0DA
:1000E00000C020F001C021F002C022F003C023F0C4
:1000F00004C024F0A0A280EF00F0A1B2F6EF00F05F
:1001000020C000F021C001F022C002F023C003F0A3
:1001100024C004F01F8E1EC0E9FF19C0EAFF1AC0F8
:10012000E1FF1BC0E2FF1CC0D9FF1DC0DAFF25C0E4
:10013000F3FF26C0F4FF27C0FAFF1100B051070BF0
:10014000006EB031016E013201321F0E01160150F6
:10015000B225E96E000EB321EA6E016A012A002A77
:1001600001D00136002EFDD7B15303E00150EF124C
:1001700003D0011E0150EF16000C606AD890603465
:10018000036A4D0FE96E000E0320EA6EECCF8FF08C
:10019000ED52EFCF8EF08EC0B0F0010EB16F0F0EAA
:1001A000B36F890EB26FCADF8EC0B0F0B16B0F0EA5
:1001B000B36F920EB26FC2DFD8906034036A320F11
:1001C000E96E000E0320EA6EECCF8FF0ED52EFCF18
:1001D0008EF08FC0B3FF8EC0B2FFA0829E90D10E72
:1001E000CF6E9C0ECE6E9E903AEF00F0D8906034A9
:1001F000036A4D0FE96E000E0320EA6EECCFAFF0FC
:10020000ED52EFCFAEF0AEC0B0F0B16B0F0EB36FEA
:10021000890EB26F93DFAEC0B0F0B16B0F0EB36F4B
:10022000920EB26F8BDF602A5F50605C03E1A09298
:10023000A19230D0D8906034036A4D0FE96E000E61
:100240000320EA6EECCFAFF0ED52EFCFAEF0AEC0D0
:10025000B0F0010EB16F0F0EB36F890EB26F6EDF8B
:10026000AEC0B0F0B16B0F0EB36F920EB26F66DF1F
:10027000A192D8906034036A320FE96E000E032019
:10028000EA6EECCFAFF0ED52EFCFAEF0AFC0B3FF00
:10029000AEC0B2FFA19280EF00F08E0E006E97C04C
:1002A00001F096C002F0036A015209E102C001F0B8
:1002B000026A080E005E015202E1006A08D0D8907E
:1002C00001BE04D0023601360006F9D7019E000CAB
:1002D000A251D8B471D0006EA651D8B46DD000260A
:1002E00004E3810E002668E204D07F0E005E64E322
:1002F00063E0A3C0AAF0A751AA1BA38FA78FA551A3
:10030000A903F4CFACF0A451A803F4CF03F0F3CFCA
:10031000ABF0A903F350AC27F450AB23000E03223B
:10032000A551A803F350AC27F450AB23000E026A8A
:1003300003220222A351A903F350AB27F450032256
:10034000000E0222A351A803F3500326F450022208
:10035000000E016A0122A551A703F350AB27F45008
:100360000322000E02220122A451A703F350032608
:10037000F4500222000E0122A351A703F3500226DB
:10038000F4500122002A01BE05D0AB3703360236F5
:1003900001360006000EABAF0AD0032A022201226A
:1003A000015005E1025003E1035001E1002AAABF18
:1003B000018EAAAF019E04D0006A016A026A036A34
:1003C000000C9A51D8B4A5D0A66F9E51D8B4A1D034
:1003D000A65F05E37F0EA627D8B09BD006D0810E7E
:1003E000A65FD8A096D0D8B494D0A6C000F0016A79
:1003F000026A036AA56B9BC0A4F0A48F9CC0A3F003
:100400009DC0A2F0190EA66FA151A25F0DE2010ED0
:10041000A35F0AE2A45F08E2A55F06E2A52BA42B76
:10042000A32BA151A22728D0A051A35F12E2010E55
:10043000A45F0FE2A55F0DE2A52BA42BA051A3277B
:10044000A151A22719E3A32B17E1A42B15E1A52B9A
:1004500013D09F518009A45F0EE2010EA55F0BE24D
:10046000A52B9F518009A427A051A327E9E3A42B22
:10047000E7E1A52BE5D70380A62F01D00BD0D890BC
:10048000A237A337A437A537D890033602360136F2
:10049000A737BAD7A7A106D0D890013202320332CB
:1004A000A73302D0000635E0A7BF1ED0D890A237F0
:1004B000A337A437A537A151A25F07E2010EA35FBE
:1004C00004E2A45F02E2A55F1AE3A051A35F05E284
:1004D000010EA45F02E2A55F12E39F518009A45FB1
:1004E00003E2010EA55F0BE3032A09E1022A07E1FB
:1004F000012A05E1002A0DE00132023203329BC0DD
:10050000A6F09F51A61BA6AF02D0018E06D0019E79
:1005100004D0006A016A026A036A000C800ED8B235
:10052000A31BA86BA96B9FC0A7F0A351A71B9E514B
:10053000D8B4DCD0A66F006EA251D8B4E0D0A65FCC
:10054000D8B481D03DE3A3C0ACF0AC8FA4C0ABF075
:10055000A5C0AAF0A96BD890AC33AB33AA33A933AA
:10056000A62FF8D7A7AF03D0A881DDD0A891A69178
:10057000A889EA6AA10EE96EE9D0A899A7BF0AD0B6
:10058000A6A113D0AC33AB33AA33A933002AD8B415
:10059000C5D00BD0ACBF0CD0D890A937AA37AB3799
:1005A000AC370006D8B4BAD0F5D7A88D6BD0A89DCB
:1005B0009FC0A7F09FAF02D0AC8FA9D0AC9FA7D0AF
:1005C000A2C0A6F0A2C000F09E51A65F9FC0ACF0F2
:1005D000AC8FA0C0ABF0A1C0AAF0A96BD890AC338F
:1005E000AB33AA33A933A62FF8D7A7AF03D0A8837C
:1005F0009AD0A893A691A88BEA6AA50EE96EA6D018
:10060000A89BA7BF0AD0A6A113D0AC33AB33AA33A3
:10061000A933002AD8B482D00BD0ACBF0CD0D8906C
:10062000A937AA37AB37AC370006D8B477D0F5D79F
:10063000A88F28D0A89FA3C0A7F0A3AF02D0AC8FEB
:1006400066D0AC9F64D0A3C0ACF0AC8FA4C0ABF0BC
:10065000A5C0AAF0A7AF04D0AC9FA88564D0A89588
:10066000A96BA691EA6AA10EE96E70D0A7BF1CD053
:100670009FC0A7F0A6A106D0AC33AB33AA33A933F1
:10068000002A4CE0A9AF0BD0AA2B09E1AB2B07E164
:10069000AC2B05E1AC33AB33AA33002A3FE0A8BD55
:1006A00086D7A8BFC7D71CD0800EAC1BACAF04D078
:1006B0003AD0A3C0A7F00AD09FC0A7F0AC5306E180
:1006C000AB5304E1AA5302E1006A21D0ACBF08D0C9
:1006D000D890A937AA37AB37AC37002EF7D71ED042
:1006E000A7AF02D0AC8F13D0AC9F11D0A2C000F046
:1006F000A3C0ACF0A4C0ABF0A5C0AAF008D09EC0C7
:1007000000F09FC0ACF0A0C0ABF0A1C0AAF0ACC09C
:1007100001F0ABC002F0AAC003F034D0006A016A55
:10072000026A036A2FD0A96BAA1FAB1FAC1FA91FB7
:10073000A92B05E1AA2B03E1AB2B01E1AC2BA8B15E
:1007400015D7A8B356D7A8B58AD7B3D7EF50AA27DD
:1007500005E3AB2B03E1AC2BD8B4A681ED52EF50EF
:10076000AB2703E3AC2BD8B4A681ED52EF50EFBE1C
:1007700001D0800AAC27D8B0A681A8B9FED6A8BB04
:100780003FD774D7000C8E0E006EA251005EA3C03E
:1007900002F0A4C001F0028E005209E0D89002528B
:1007A00002E1015204E002320132002EF7D7A3AF7A
:1007B00005D0011E021E012AD8B4022A000C976B34
:1007C00095C096F06ADD03C0A5F002C0A4F001C098
:1007D000A3F000C0A2F06F0EA96F120EA86F030E57
:1007E000A76F750EA66F74DD00C096F001C097F07C
:1007F00002C098F003C099F003C09DF002C09CF0C5
:1008000001C09BF000C09AF0A16BA06B7F0E9F6FA0
:10081000860E9E6FD6DD00C09AF001C09BF002C02C
:100820009CF003C09DF0D89203C0A1F002C0A0F0DC
:1008300001C09FF000C09EF06F0EA56F120EA46F56
:10084000030EA36F750EA26F69DE00C09EF001C09B
:100850009FF002C0A0F003C0A1F003C0A5F002C049
:10086000A4F001C0A3F000C0A2F0800EA96F960E04
:10087000A86F180EA76F930EA66F2ADD03C0A5F010
:1008800002C0A4F001C0A3F000C0A2F07CDF02C04F
:1008900003F00150FF08006EFF0E035600C001F088
:1008A00003C002F0000C036A9251290FE96E000E9A
:1008B0000320EA6E91C0EFFFD8909235036A320FA1
:1008C000016E000E032201C093F003C094F091C0AA
:1008D00095F075DF94C0EAFF93C0E9FF02C0ECFF1A
:1008E000ED5201C0EFFF000C006A016A9151D890EF
:1008F00092B100260032013292B30026003201325A
:1009000092B500260032013292B700260032013241
:1009100092B900260032013292BB00260032013229
:1009200092BD00260032013292BF00260032013211
:1009300006EF05F0612A61500408D8A48FD0939C7B
:100940008A9C8E6B5F508E5DD8B085D0036A8E51C5
:10095000440FE96E000E0320EA6EEFBE38D0EF5070
:10096000000835E2036A8E51290FE96E000E03205C
:10097000EA6EEF50FF088F6F036A8E51440FE96EE5
:10098000000E0320EA6EEFCF00F000BE03D000504F
:100990008F5D18E3036A8E51290FE96E000E032064
:1009A000EA6EEFCF8FF0036A8E51440FE96E000EAE
:1009B0000320EA6EEF508F25906F916F8EC092F0FA
:1009C00072DF05D0FF0E916F8EC092F06CDF036A6C
:1009D0008E51440FE96E000E0320EA6EEFBE01D087
:1009E00038D0036A8E51290FE96E000E0320EA6E9B
:1009F000EFCF8FF0036A8E51440FE96E000E032093
:100A0000EA6EEFCF91F0FF0E926F6ED701C000F04B
:100A100001BE08D08F51005C05E3916B8EC092F04F
:100A200042DF17D0036A8E51290FE96E000E0320B2
:100A3000EA6EEFCF8FF0036A8E51440FE96E000E1D
:100A40000320EA6EEF508F25906F916F8EC092F069
:100A50002ADF8E2B77D7616A939C8A8C9E92CC6A10
:100A60009E923AEF00F070C05FF0606A716A705059
:100A7000715C32E2D8907134036A6E24E96E6F5073
:100A80000320EA6EECCF73F0ED52EFCF72F07252AA
:100A900002E173521FE0D8907134036A4D0F016E6A
:100AA000000E032203C073F0D8907134036A6E24E1
:100AB000E96E6F500320EA6EECCF03F0ED52EFCFFA
:100AC00074F073C0EAFF01C0E9FF03C0ECFFED5210
:100AD00074C0EFFF712ACBD7716A5F50715C36E248
:100AE000036A7150290FE96E000E0320EA6E7F0E33
:100AF000EF6ED8907134036A320F016E000E03223C
:100B000001C072F003C073F0036A7150290FE96EDF
:100B1000000E0320EA6EEFCF74F0186AF2BC188C56
:100B2000F29CF2BE188EF29E74C095F048DE18BC9E
:100B3000F28C18BEF28E73C0EAFF72C0E9FF02C0E9
:100B4000ECFFED5201C0EFFF712AC7D7780E0609FE
:100B5000CA6E7D0ECB6ECF6ACE6A616AB50ECD6E5F
:100B6000D10ECF6E9C0ECE6EB150480BA509B16E62
:100B70009D809D82A092C00EF21228EF06F0036ABB
:100B80006F50440FE96E000E0320EA6E6EC0EFFF57
:100B9000000CF86A9F909F92A282D08E0D8EEA6A16
:100BA000E96A0A0EAF6EA60EAC6E900EAB6EC180F7
:100BB000C182C184C196296A2A6A2B6A2C6A2D6A6D
:100BC0002E6A2F6A306A316A326A336A346A356A49
:100BD000366A376A386A396A3A6A3B6A3C6A3D6AF9
:100BE0003E6A3F6A406A416A426A436A446A456AA9
:100BF000466A476A486A496A4A6A4B6A4C6A4D6A59
:100C00004E6A4F6A506A516A526A536A546A556A08
:100C1000566A576A586A596A5A6A5B6A5C6A5D6AB8
:100C20005E6A5F6A080E626E7C0E636E090E646E09
:100C30007C0E656E120E666E7C0E676E150E686E0B
:100C40007C0E696E6F6A620E6E6E040E706E0BD74C
:100C50009EAAFED7AECF6AF09EAAFED7AECF6BF0AB
:100C60009EAAFED7AECF6CF09EAAFED7AECF6DF097
:100C70006AC06EF06F6A83DF6BC06EF0010E6F6E3C
:100C80007EDF186AF2BC188CF29CF2BE188EF29EBF
:100C90006CC091F0020E926F06DE18BCF28C18BE8A
:100CA000F28E186AF2BC188CF29CF2BE188EF29E7C
:100CB0006DC091F0030E926FF6DD18BCF28C18BE79
:0E0CC000F28E590E9EA8FED7AD6EC2D703006D
:020000040030CA
:0E00000000220E0E000181000FC00FE00F4025
:00000001FF
